:020000001028C6
:10000800FE00030EF0000408F1000A08F200831253
:1000180003137F08F3006729722983120313AD00C5
:10002800872187217908013A83120313AC002C0831
:10003800F9007908013A031D222823282528872159
:10004800272884212728043083120313AC002C08A6
:10005800AE002E08FF3A031D3228332835285428CD
:1000680054287608840083130008AC002E0A3E2822
:100078000310AC0CFF3E031D3C282C1C44284528CB
:1000880047288721492884214928013083120313EE
:10009800AE022E08FF3A031D52285328352854284B
:1000A8000530AC002C08AE002E08FF3A031D5D2871
:1000B8005E2860287F287F282D0884008313000885
:1000C800AC002E0A69280310AC0CFF3E031D6728FC
:1000D8002C1C6F2870287228872174288421742882
:1000E800013083120313AE022E08FF3A031D7D2848
:1000F8007E2860287F284721080083120313AC005C
:10010800AD010330F4007408AE002E08FF3A031D59
:100118008E288F289128DF28DF28FF3086000130BD
:10012800F4002E0A99280310F40DFF3E031D9728AA
:100138007408FF3AF500750886050430F400740861
:10014800AF0008302F02031CAA28AB28AD28D628F8
:10015800D6280130F4007408AD070608F4002F0A09
:10016800B7280310F40CFF3E031DB5287418BD28EA
:10017800BE28CB282D08F4002C08840074088313AB
:1001880080000130AA000030AB00DF28DF280130F2
:10019800F4007408AF0708302F02031CD428D528B0
:1001A800AD28D6280130AE022E08FF3A031DDD28FF
:1001B800DE289128DF28080083120313B301B20157
:1001C80002308316031381000730831203139F0044
:1001D800831603138501F03086008B1783120313EF
:1001E8001F149F141F158501FF3086001D30B000B5
:1001F8003008B2008B018B15B10104290429630072
:100208000B1C0729082903290929FF308312031326
:100218008600333081200130831203132A062B0411
:10022800031D1729182904293230B0003008F600B8
:100238003330112083120313AA01AB01B101031457
:10024800B10D0429042904291028F5018312031388
:1002580005140514051405140510051005100510DE
:1002680005100510051005100510051005100130C2
:10027800F4007408F50720307502031C4429452949
:100288002A2905100800A001A201A4017430A200C7
:100298000230A0000130A400A00B5029A20B502965
:1002A800A40B50290800F50183120313051001302F
:1002B800F4007408F5073C307502031C64296529AD
:1002C8005829662908007308FF0072088A00710817
:1002D8008400700E8300FE0E7E0E0900F701F801FF
:1002E800F9018313203084002C307C218301E0281D
:1002F80064008001840A04060319003404067D2979
:0C03080029215721080057212921080055
:02400E0001FFB0
:00000001FF
